:1000000000308A0036280000831A0A28A400030E54
:10001000A5000F288312A400030EA500A5140A084A
:10002000AB008A018313A40E0408A6002008A700D1
:100030002108A8002208A9002308AA0083120B1E89
:1000400023288B183C28260884002708A0002808AD
:10005000A1002908A2002A08A3002B088A00250E67
:1000600083008312240EA51883160900FF2383162C
:10007000900000308A009A280B122C1C41282C106A
:1000800042282C140B168B108A1123288316051274
:10009000831205161A30A000A00B4C28000083160E
:1000A00085128312851683160512831205121A30E3
:1000B000A000A00B59280000831685128312851218
:1000C0001A30A000A00B6228000008002E30840027
:1000D0000008031979280130A100A001A00B6E28A7
:1000E000A10B6D284A30A000A00B74287728800B44
:1000F0006B28080083168512831285161A30A0001B
:10010000A00B8028000083160512831205168316A3
:100110008512831285121A30A000A00B8D280000D2
:1001200083160512831205121A30A000A00B962820
:100130000000E32884011F3083052C104130AD00FE
:10014000AC101F1383161F109F101F119F11073033
:10015000831299001F1383161F109F101F119F11E8
:100160001F129F121F1383129F131F14831601085F
:10017000C73908388100831290010730990083162F
:100180000508850003308312A000A00BC5281908BC
:100190008C118316990183120B16C0308B048316C1
:1001A0000113851583128519DD2846202D08AE0020
:1001B0006620AC148316D12883122C1CEE28AC1CAC
:1001C000EE280B127A282D08AE00662083168515BE
:1001D0008312851DEC28AC100B16DD282C18FF2887
:1001E000AC18FF280B1246202D08AE00662083169F
:1001F00085158312851DFD28AC140B16EE28DD280D
:02020000630099
:02400E00043F6D
:00000001FF
